:020000040000FA
:10000000831285010730990083169F012C308500EB
:100010008312FF30850005303020553027205230C4
:100020001B20122800308500133030200D3027208F
:1000300068301B200928F13EA00020181F28A018B6
:100040002128A0182328FC3E031823280800FF3E7F
:10005000A1005E301B2060301B20A10B2B28080064
:10006000FF3EA200633027205D301B206330272035
:100070005F301B20A20B362808004120422042207E
:0C00800041204220452000000000080044
:02400E00D33F9E
:00000001FF
